:10000000020BBEAAAAAAAAAAAAAAAA020EFBAAAA76
:10001000AAAAAA020E76AAAAAAAAAA0208B8AAAAF4
:10002000AAAAAAAAAAAAAAAAAAAAAA020B31AAAAF0
:10003000AAAAAA020FDEAAAAAAAAAAAAAAAAAAAA2F
:10004000AAAAAA020800AAAAAAAAAA02069DAAAA5D
:10005000AAAAAA020800AAAAAAAAAAAAAAAAAAAAF4
:10006000AAAAAAAAAAAAAAAAAAAAAAAAAAAAAAAAF0
:10007000AAAAAAAAAAAAAAAAAAAAAAAAAAAAAAAAE0
:1000800090E6B9E0700302015B14700302020424DD
:10009000FE700302029924FB7003020155147003E1
:1000A00002014F147003020143147003020149243A
:1000B000056003020305120FE6400302031190E6F8
:1000C000BBE024FE602C14604724FD6016146031F0
:1000D00024067065E52490E6B3F0E52590E6B4F0DB
:1000E000020311E52C90E6B3F0E52D90E6B4F002A2
:1000F0000311E52690E6B3F0E52790E6B4F002039D
:1001000011E52890E6B3F0E52990E6B4F00203117A
:1001100090E6BAE0FF120ECFAA06A9077B01EA49D2
:10012000600DEE90E6B3F0EF90E6B4F002031190AC
:10013000E6A0E04401F002031190E6A0E04401F0E3
:10014000020311120FA7020311120FD6020311129C
:100150000FCE020311120F95020311120FE8400394
:1001600002031190E6B8E0247F602B14603C240267
:1001700060030201FAA200E433FF25E0FFA204E4D9
:10018000334F90E740F0E4A3F090E68AF090E68BDE
:100190007402F0020311E490E740F0A3F090E68AC5
:1001A000F090E68B7402F002031190E6BCE0547EFE
:1001B000FF7E00E0D3948040067C007D0180047CBB
:1001C000007D00EC4EFEED4F24C4F582740F3EF529
:1001D00083E493FF3395E0FEEF24A1FFEE34E68F36
:1001E00082F583E0540190E740F0E4A3F090E68AC2
:1001F000F090E68B7402F002031190E6A0E0440157
:10020000F0020311120FEA400302031190E6B8E076
:1002100024FE601D2402600302031190E6BAE0B4DC
:100220000105C20002031190E6A0E04401F00203C0
:100230001190E6BAE0705990E6BCE0547EFF7E0073
:10024000E0D3948040067C007D0180047C007D002A
:10025000EC4EFEED4F24C4F582740F3EF583E4931B
:10026000FF3395E0FEEF24A1FFEE34E68F82F583A5
:10027000E054FEF090E6BCE05480FF131313541FCB
:10028000FFE0540F2F90E683F0E04420F0020311CA
:1002900090E6A0E04401F08078120FEC507390E6F5
:1002A000B8E024FE60202402706790E6BAE0B40152
:1002B00004D200805C90E6BAE06402605490E6A04C
:1002C000E04401F0804B90E6BCE0547EFF7E00E00D
:1002D000D3948040067C007D0180047C007D00EC8E
:1002E0004EFEED4F24C4F582740F3EF583E493FF78
:1002F0003395E0FEEF24A1FFEE34E68F82F583E034
:100300004401F0800C120FEE500790E6A0E044018B
:10031000F090E6A0E04480F022E4F517F516F5151C
:10032000F514C205C200C204C201120A9D7E0A7FF2
:10033000008E248F25752C0A752D1275220A7523BF
:100340001C752A0A752B43752F0A753071EE54E01F
:10035000700302045D7518007519808E1A8F1BC317
:10036000749B9FFF740A9ECF2402CF3400FEE48F5B
:10037000138E12F511F510F50FF50EF50DF50CAF06
:1003800013AE12AD11AC10AB0FAA0EA90DA80CC381
:10039000120E105026E519250FF582E518350EF5D9
:1003A0008374CDF0E50F2401F50FE4350EF50EE46E
:1003B000350DF50DE4350CF50C80C4E4F50FF50EA4
:1003C000F50DF50CAF13AE12AD11AC10AB0FAA0EBC
:1003D000A90DA80CC3120E105031AE0EAF0FE51BC5
:1003E0002FF582E51A3EF583E0FDE5192FF582E54C
:1003F000183EF583EDF0EF2401F50FE43EF50EE431
:10040000350DF50DE4350CF50C80B98518248519EA
:100410002574002480FF740A34FFFEC3E52D9FF588
:100420002DE52C9EF52CC3E5279FF527E5269EF5A7
:1004300026C3E5299FF529E5289EF528C3E5239FD6
:10044000F523E5229EF522C3E52B9FF52BE52A9E99
:10045000F52AC3E5309FF530E52F9EF52FD2E8430E
:10046000D82090E668E04409F0E04402F090E65EAF
:10047000E0440CF043E80443E80290E6507404F0D2
:10048000000000E4F5B290E67AF043B288F58043CC
:10049000A82E438804438910758B6F758DFE90E6F6
:1004A0008F04F075AF07759DE1E4F59E90E65CE082
:1004B000443DF0D2AF90E680E020E105D207120E75
:1004C0004790E680E04408F00000000000000000D3
:1004D00000E054F7F0538EF8C20530010512008099
:1004E000C201300529120FE25024C2051207DB2099
:1004F000001690E682E030E704E020E1EF90E6822B
:10050000E030E604E020E0E4120EA3120FE4120F44
:10051000F080C7C0E0C0F0C083C082C0D075D000FA
:10052000C000C001C002C003C004C005C006C007AF
:10053000759AE7759B80759DE130060302061A7572
:100540000A00750B0090E67BE0FF7432250BF8A6DD
:1005500007050BE50B7002050AE59B2480C3940692
:1005600040E3E532120E2105F900058908059F10C8
:1005700005DF2005B93005D240061250060A600595
:10058000DACC05CCFF0000061A159B5391EF90E6DC
:100590005F7408F090E68DE4F0120D670206827435
:1005A000FD259BF59B5391EF90E65F7408F090E674
:1005B0008DE4F0120D6702068290E7C0740AF0A382
:1005C000E580F090E68F7402F00206745380F70223
:1005D000067490E68F7401F08040753900803B907E
:1005E000E7C074DDF0A37431F0A3742EF0A3743669
:1005F000F090E68F7404F0807B53A8F785368A75F7
:10060000CDFE75CC6F759E00801090E618740DF0CD
:10061000806290E618740CF0805A90E67BE090E6D9
:100620007CF0E59B2480FF90E68DE0FEEFC39E40CA
:10063000E9E53324FEFFE59EC39F5006E4F0D206B1
:100640008032C206759DE1759E00438902758E0059
:10065000858A8C75C800E5367006E53542808005D0
:10066000E535F4528043800890E67CE0F538438815
:100670001043C8045391EF90E65F7408F090E68D44
:10068000E4F0D007D006D005D004D003D002D001CA
:10069000D000D0D0D082D083D0F0D0E032C0E0C043
:1006A00083C082C0D075D000C000C004C005C006A1
:1006B000C0075391DF90E678E05404FF7E003002DB
:1006C0000BE0F430E1067C007D0180047C007D00BD
:1006D000EC4EFEED4F4E6008E4FF12096F0207C8B2
:1006E000E53224F860030207C8E53314604904606A
:1006F000030207C8E59B2480FFBF050B059B90E61E
:1007000079E534F00207C8E5372406FFE433FEAD8F
:100710009BED2480FDE434FFFCC3ED9FEE6480F884
:10072000EC648098500B90E67BE090E679F002074D
:10073000C81209660207C8E536701CE59B2480C311
:100740009406500B059B90E679E534F00207C875D6
:100750003601120D67807130020F90E679E075085E
:1007600000F509C202059B805FE5372406FFE433EC
:10077000FEAD9BED2480FDE434FFFCC3ED9FEE64F1
:1007800080F8EC648098503DE5372405FFE59B2414
:1007900080B5071490E678E04440F090E679E09068
:1007A000E67BF07F0112096FE5372404FFE59B2407
:1007B00080B5070790E678E04420F090E679E09075
:1007C000E67BF08003120966D007D006D005D0047E
:1007D000D000D0D0D082D083D0E03290E682E04406
:1007E000C0F090E681F04387010000000000227411
:1007F00000F58690FDA57C05A3E582458370F9226E
:10080000020F3900020F7F00020F6900020F510032
:10081000020DA200020DD900020FF100020FF2003A
:10082000020FF300020FF400020C4A00020513004D
:10083000020FF500020FF600020FF700020FF8009A
:10084000020FF900020FF200020FFA00020FFB0084
:10085000020FFC00020FFD00020FFE00020FFF005E
:1008600002100000020FF200020FF200020FF2006D
:100870000210010002100200021003000210040026
:10088000020F1C00021005000210060002100700F3
:10089000021008000210090002100A0002100B00EA
:1008A00002100C0002100D0002100E0002100F00CA
:1008B0000210100002101100C0E0C083C082C0D03E
:1008C0005388BF758B6F758DFEE59EC3947A507209
:1008D000300313E58020E10E43800890E67CE53884
:1008E000F0753800C203200313E58030E10E538019
:1008F000F790E67CE538F0753800D203E538F470FF
:100900003AE59EC3947A503390E67CE538F075382A
:1009100000E4F00521E52194004020E59E94185064
:100920001A759E00752100753800B2035388BF7593
:100930003D0090E65EE04404F080224388400538A4
:10094000801B53A8F75388F75388BF753800C2033C
:10095000752100753D0290E65EE04404F0D0D0D0F1
:1009600082D083D0E03290E678E04440F07F01EF1F
:1009700014603E0460030209FF90E7C074FFF0A317
:10098000E59BF090E678E090E7C2F090E678E0F43E
:1009900030E604E04440F0E490E679F00000000026
:1009A000000090E678E090E7C3F090E68F7405F0E1
:1009B00022E533700D90E7C07410F090E68F74015B
:1009C000F022759B80759DE7759EC090E67BE09058
:1009D000E67CF0E5372406FFE433FEAD9BED248092
:1009E000FDE434FFFCC3ED9FEE6480F8EC64809876
:1009F00040D9E537240690E68FF05380F7D20222E3
:100A00001201000200000040470502100000010230
:100A100000010A0600020000004001000902270050
:100A2000010100A0320904000003FF0000000705D7
:100A30000102400000070581024000000705820214
:100A400000040009022E00010100A0320904000088
:100A500004FF000000070502024000000705040231
:100A6000400000070586024000000705880240009C
:100A7000000403090410034E00650078007400634D
:100A8000006F006D001603480044002D0055005310
:100A90000042002000440056005200000090E60B87
:100AA0007403F000000090E6047480F0000000740D
:100AB00002F000000014F0000000E4F000000090DC
:100AC000E6007412F090E6017443F090E61074A012
:100AD000F090E68D7401F090E61174A0F090E618A5
:100AE000740DF090E6137420F090E614F090E61583
:100AF000F090E61274E8F0E490E602F00000009056
:100B0000E603F090E670F090E609F000000090E651
:100B1000207404F0000000E490E621F00000009052
:100B2000E630749AF0000000E490E631F000000036
:100B300022C0E0C083C082C0D053C8FBE538D39444
:100B400000400D75CDFE75CC6F153843C80480622A
:100B5000E59EC39533502790E67CE0F538E5883074
:100B6000E40AE535F452805388EF8007E53542808A
:100B700043881075CDFE75CC6F43C8048034759ED4
:100B800000E537B47719753700759DE1059E753816
:100B90000075CDFE75CC6F43881043C80480135395
:100BA00088EF53C8FB90E68DE4F0E535F4528043BE
:100BB000A80853C87FD0D0D082D083D0E032787FCD
:100BC000E4F6D8FD75813D020C05020319E493A3F8
:100BD000F8E493A34003F68001F208DFF48029E4EF
:100BE00093A3F85407240CC8C333C4540F4420C83B
:100BF000834004F456800146F6DFE4800B010204D2
:100C00000810204080900FB9E47E019360BCA3FFE0
:100C1000543F30E509541FFEE493A360010ECF5406
:100C2000C025E060A840B8E493A3FAE493A3F8E4F5
:100C300093A3C8C582C8CAC583CAF0A3C8C582C861
:100C4000CAC583CADFE9DEE780BEC0E0C0F0C0836A
:100C5000C082C0D075D000C000C001C002C003C0B7
:100C600004C005C006C00790E65F7404F05391EF1E
:100C7000300605120CBF802CE53D7005F59E43A89B
:100C800008438008E53D6401601AE53DB4020512A1
:100C90000CBF801090E7C074CCF0A3E539F090E66B
:100CA0008F7440F0D007D006D005D004D003D00216
:100CB000D001D000D0D0D082D083D0F0D0E0327537
:100CC0009AE720062AE490E7C0F0A3E59EF0A3741B
:100CD000A0F0A37402F0A37497F0E4A3F0759BC690
:100CE000F59E90E7C1E0D3943A400CD20680087597
:100CF0009BC0C206759E3A90E7C1E0FF90E67CE09B
:100D000090E67BF0AE9BEEC3748094815006E59E26
:100D1000C39F40E890E68F7440F05380F7E4F53DC0
:100D2000228E1C8F1D90E600E054187012E51D24E1
:100D300001FFE4351CC313F51CEF13F51D8015905E
:100D4000E600E05418FFBF100BE51D25E0F51DE59A
:100D50001C33F51CE51D151DAE1C7002151C4E60E4
:100D6000051207EF80EE2290E678E0F430E62DE001
:100D70004480F0E53224F0601C24087024E533B48C
:100D8000010CE536B4010790E67974A1F02290E6F3
:100D90007974A0F02290E679E534F022E4FF12099C
:100DA0006F22C0E0C083C08290E680E030E70E850D
:100DB0002226852327852A28852B29800C852A260B
:100DC000852B278522288523295391EF90E65D7492
:100DD00010F0D082D083D0E032C0E0C083C08290D7
:100DE000E680E030E70E852226852327852A2885A0
:100DF0002B29800C852A26852B27852228852329C7
:100E00005391EF90E65D7420F0D082D083D0E03231
:100E1000EB9FF5F0EA9E42F0E99D42F0E89C45F038
:100E200022D083D082F8E4937012740193700DA3E2
:100E3000A393F8740193F5828883E4737402936832
:100E400060EFA3A3A380DF30070990E680E0440AA7
:100E5000F0800790E680E04408F07FDC7E05120D0C
:100E60002190E65D74FFF090E65FF05391EF90E61D
:100E700080E054F7F022C0E0C083C082C0D0E59E7D
:100E8000C3947A501543884043800890E68FE4F07D
:100E900090E65EE054FBF0753D01D0D0D082D08367
:100EA000D0E03290E682E030E004E020E60B90E60D
:100EB00082E030E119E030E71590E680E04401F08F
:100EC0007F147E00120D2190E680E054FEF022A9EE
:100ED00007AE2FAF308F828E83A3E064037017AD0F
:100EE0000119ED7001228F828E83E07C002FFDECD2
:100EF0003EFEAF0580DF7E007F0022C0E0C0D0E56F
:100F000036D394004011E58055356007E535F4523D
:100F1000808004E5354280D0D0D0E032C0E0C0838C
:100F2000C0825380F77539015391BF90E651E05468
:100F3000FEF0D082D083D0E032C0E0C083C082D245
:100F4000015391EF90E65D7401F0D082D083D0E040
:100F500032C0E0C083C082D2055391EF90E65D7449
:100F600008F0D082D083D0E032C0E0C083C082538A
:100F700091EF90E65D7404F0D082D083D0E032C06F
:100F8000E0C083C0825391EF90E65D7402F0D0829E
:100F9000D083D0E03290E740E53CF0E490E68AF080
:100FA00090E68B04F0D32290E740E531F0E490E640
:100FB0008AF090E68B04F0D322C182013D00C10685
:100FC000013900000001020203030404050590E654
:100FD000BAE0F53CD32290E6BAE0F531D32253D8FB
:100FE000EF32D322D322D322D322D322D322D3222D
:100FF00022323232323232323232323232323232E1
:1010000032323232323232323232323232323232C0
:101010003232AAAAAAAAAAAAAAAAAAAAAAAAAAAA20
:10102000AAAAAAAAAAAAAAAAAAAAAAAAAAAAAAAA20
:10103000AAAAAAAAAAAAAAAAAAAAAAAAAAAAAAAA10
:10104000AAAAAAAAAAAAAAAAAAAAAAAAAAAAAAAA00
:10105000AAAAAAAAAAAAAAAAAAAAAAAAAAAAAAAAF0
